:020000040000FA
:100000002500780A2A050A040D0C2400050C2B0093
:100010004A05670066070A0A68006607160AA8020A
:100020000000680C880003070D0A010868000A0632
:10003000210A6606290AAE0C880003060208A802F7
:10004000190A6607290AAE0C880003060208A802EE
:10005000210A010CAA01220C880003070308680C7E
:1000600088000307360A2A073A0A0408020CAA0184
:100070002A06160A4A074B0A0A07430A8707A702F5
:100080009609160A09084A040C0C870003070A0897
:100090000A0C2700160AE7004306580A010C8701DC
:1000A0004307550A0A06160A07080A036903160ACF
:1000B0000A06080809022000A402EB02480A000808
:1000C0000D0C2400040C2B004000C001A402EB0224
:1000D000650A910043076D0A00080C089A0C8D0010
:1000E0004307770AE60C8E004307770A00080D08DD
:1000F0006600400006000400470C020061009B09F6
:1001000096090209FF0E43078A0A6009FF0E43079A
:100110008A0A6E09290029024307800AAF046F0684
:10012000AF05FF0C8F012600A009800AE107000837
:100130006100EC020008EA040F0C2C0066000008C5
:08014000EA050F0C2C00000879
:0401480000080008A3
:021FFE00EA0FE8
:00000001FF
